:030000000219FDE5
:03000B000200AA46
:03002B0002016C63
:03005B000202FF9F
:030073000202E5A1
:1000800002030406080C10182030406080040608A3
:100090000C10182030406080A0C000070F1F3F0DDB
:1000A0000D04050D050305030302C2AFC0D0C0E077
:1000B000206217E5256002E473E525F4F58A758B67
:1000C00000D262D0E0D0D0D2AF3285268AC262E5BB
:1000D00026F4603C306803207210758B00D0E0D0AD
:1000E000D0C283C294C295D2AF32C283C294C295A9
:1000F000206E13206610740CD5E0FDE57EB5070474
:10010000429021064280758B00D0E0D0D0D2AF3231
:10011000758A00C28DD262210601B9306805206659
:1001200002D28301B9306805206602D29401B93049
:100130006805206602D29501B9C28030680A20663F
:10014000077408D5E0FDD28301B9C28230680A2065
:1001500066077408D5E0FDD29401B9C29730680AE9
:100160002066077408D5E0FDD29501B9C2AFC2ADD3
:1001700053E6EFC0D0C0E0D2D3D2AFC2CEE52A6002
:1001800007207449152A21CD7800790020742EE5C6
:1001900080307E01F430E50278FF53DACF207E0311
:1001A00043DA20307E0343DA10C2D8C271E58030D2
:1001B0007E01F430E50279FFC3E89970CB3061032A
:1001C000752A18207403752A18885FD27020740D60
:1001D000E52B6004152B21DD43DA01C2D820700223
:1001E000413BA85F206102C2702074367982B70457
:1001F00031C3E894F0400374F0F8E8C4540F28F8D1
:100200007984B703024122C313C313872120080254
:10021000C313200A06C3C898F8412228F850037473
:10022000FFF88822E52D54066011E533C313C3138C
:1002300024062522F52250037522FF7882B6045940
:10024000852224A824C3E52495644002A864C3E859
:1002500095664002A8668825E5697002418CC3E86E
:10026000AA699A5003E8FAE4F9EAC333FBE56BF4B0
:100270005B29400D256AF8E56A6002156A400B416A
:100280008C0AC3E56A9A5002056A78FF8826C26E16
:10029000C3E52694F84002D26EC3E525944040029F
:1002A000D26420CF0AD0E0D0D043E610D2AD32C223
:1002B000CF053A7801E52A6005307402152AC3E5B6
:1002C0005F9401400575620041DB756300756C0049
:1002D000E5622401F56250037562FFD0E0D0D0439F
:1002E000E610D2AD32C2AFC0D053E67FC260759186
:1002F00000855694855795759104D0D0D2AF32C2FF
:10030000AF53E6EFC2ADC0D0C0E0C0F0D2D3D2AFA1
:10031000A8FBA9FCC2D8307102616653DACF207EF7
:100320000343DA10307E0343DA20D271E580307E59
:1003300001F420E502613D88278928A19353DACF93
:10034000207E0343DA20307E0343DA10C2D8C27124
:10035000307402A17F7800E580307E01F430E50240
:10036000A17F885FA16753DACF207E0343DA203074
:100370007E0343DA10C271206102813F53DACF203D
:100380007E0343DA10307E0343DA20C2D8D271886C
:100390005A895BC3E89558F8E99559F97B007E08BE
:1003A0007A00C3E8948CE994005005755E008131B1
:1003B000882178A2E6A8216055C3E894C8E9940092
:1003C0005008E4D2E4FB7A0A810CC3E89468E9940B
:1003D000015008E4D2E3FB7A0F810CC3E894D0E922
:1003E00094025008E4D2E2FB7A1E810CC3E894A088
:1003F000E994055008E4D2E1FB7A3C810CC3E8940F
:1004000098E994085008E4D2E0FB7A787E00C3E8CB
:10041000955CFCE9955DFD30E70AECF42401FCED08
:10042000F43400FD755E00C3EC9AED9E5003755EDA
:1004300001885C895D855A58855B597802A167C33C
:10044000E89527F8E99528F9307C02A14B307B022A
:10045000A14B307A02A1442075028162E9FDE8FCDB
:100460008181E9C313F9E813F8307902A144E9C3A3
:0F04700013F9E813F8307802A144E9C313FDE84B
:10047F0013FC20612CC3EC941CED94024002819874
:10048F00ED701EC3EC94C850180529E529700215AC
:10049F0029C3E529940A5002A17F755F00D270A18C
:1004AF007FE529600215297888E6F97400207F0816
:1004BF007896B90302789EE624FAFEE43400FFC36F
:1004CF00EC9EFCED9FFD9208B90310A20850072087
:1004DF007609D27681EA307602C276A2085016B932
:1004EF00030DECF42401FCEDF43400FD0205047857
:1004FF00007900A14BB90315EC33FCED33FDC3ECD0
:10050F00940AFCED9400FD50047C007D00C3EC9434
:10051F00FFED9400400678FF7900A14BEC8575F054
:10052F00A4C5F0A2F733F87900400302056778FFFE
:10053F007900020567E9C313F9E813F8307C0EE977
:10054F00600278FFC3E81338F8E43400F9C3E89485
:10055F00FFE99400400278FF885FD270206102A10A
:10056F007F741FF4552F4BF52FC274EB7002D274AA
:10057F00752A18307403752A0A306102A19320740A
:10058F000353DAFE207403752B06D0F0D0E0D0D0E1
:10059F00D2AD43E6103279010205C379030205C3D8
:1005AF00790A0205C3791E0205C379640205C3796E
:1005BF00C80205C37817E4D5E0FDD8FAD9F6227A38
:1005CF00147B780205EA7A107B8C0205EA7A0D7BA0
:1005DF00B40205EA7A0B7BC80205EA7902B27DE420
:1005EF00C282D5E0FDD294D5E0FDC294D5E0FDD214
:1005FF0082D5E0FDD283E576D5E0FDC2837496D532
:10060F00E0FDD9D9EAF8D5E0FDD8FBDBCEC28222D6
:10061F00C37C007D0075F00005F0EA33FAEB33FB85
:10062F0050F6EB13FBEA13FAC3E9FFE8FEE89AF87A
:10063F00E99BF95004EFF9EEF8B3EC33FCED33FD21
:10064F00D5F0DFEDF9ECF822E889F08A20D2D4F862
:10065F00A9F07B0030F70B7BFFF42401F8E9F434A9
:10066F0000F9E88520F0A4ADF0F8E98520F0A4AFFB
:10067F00F0FEED2EF974003FFA7C04C3EA13FAE999
:10068F0013F9E813F8DCF48BF030F70AE8F42401DF
:10069F00F8E9F43400F9E889F0C2D4F8A9F0227827
:1006AF0082B60403020709C3E55F94014003020603
:1006BF00D3852224E4F545F546F547F548F549C2BB
:1006CF006D0207097882E6FCD26DE522F5237838B2
:1006DF0079C7AA40AB41C3EB13FBEA13FAEC1460E2
:1006EF0013C3EB13FBEA13FAEC14146007C3EB13F9
:1006FF00FBEA13FAD11F8845894622C3E5459523A6
:10070F00F8E5469400F9500CC3E89480E994FF4053
:10071F001602073AC3E8947FE99400500302073AA0
:10072F00787F790002073A788079FF884A894B22CF
:10073F00E54A2547F8E54B3548F9854B20E4300766
:10074F0001F43549FA30E709C3EA94F0401502077E
:10075F0078C3EA940F500302077878FF79FF7A0F76
:10076F00020778780079007AF0C3E5249564500A7F
:10077F00C374019524500B020796E54B20E70E0238
:10078F000796E54B30E706884789488A492278A4BF
:10079F00E6FAC3E54A33F8E54B33F9D157E930E7C9
:1007AF000BC3E89480E994FF4013E1D0C3E8947F32
:1007BF00E994005002E1D0787F7900E1D078807918
:1007CF00FFE820E715C3E52398F84009C3E8940133
:1007DF0040030207F778010207F7E8F42401252305
:1007EF00F840030207F778FF884C2278A5E6FAA8AD
:1007FF0048A949120657E930E70CC3E89401E99478
:10080F00FF401602082CC3E894FFE994005003023E
:10081F00082C78FF790002082C780179FFE920E78E
:10082F0015C3E54C98F84009C3E89401400302084A
:10083F00537801020853E8F42401254CF8400302D1
:10084F00085378FF88242278FFC26420693D206A0C
:10085F0012D264C3E541940A4009C3E52594405080
:0E086F0002C26479A1E76023E541601F74FFB7
:10087D008541F0848539F0306A0375F005A4F8C51B
:10088D00F0600278FFC3E895675002A8678866227A
:10089D00C3E5409440E5419401E56650031401AE73
:1008AD00046002F566220208B62275E8902278836C
:1008BD00E6FFE5E820ECF7A8BDA9BE0573C3E57317
:1008CD0094084052757300E9FA79A0E76044EA7024
:1008DD0007E574601B0208F1C3E895746010E574B8
:1008ED005006600C140208FD0460F90208FDE57461
:1008FD00F574C3946D401B7564C0C39404401375A7
:10090D006480C39404400B756440C3940440037524
:10091D00640075BB0922E5642410500274FFF56470
:10092D007982B70402214AC3A864E524985002A82D
:10093D0024C3E895664002A86688258826E573B429
:10094D00070375BB1022743279A687F0A4C5F0A2F7
:10095D00F733F8C3E895644002A864882288248898
:10096D002588268867227540007541F022C2AF7533
:10097D00C820A8CCA9CDAA3A30CF010A75C824D277
:10098D00AFAB3BAC3C883B893CC3E89BF8E99C2072
:10099D006908F9306702418F21ECAD3D8A3DF9EAD6
:1009AD009DFA600478FF79FFAE3EAF3F8B3E8C3FE2
:1009BD00C3EC9FFCC3E99CF542A83BA93CC3E89E50
:1009CD00F8E99FF9C3E54113FBE54013FAE82AF571
:1009DD0040E93BF54150067540FF7541FF4136AA90
:1009ED0040AB41AC40AD417E047F02C3EB9404406B
:1009FD00021E1FC3EB940840021E1FC3ED13FDEC36
:100A0D0013FCDEF7C3EA9CFAEB9DFBEF6009C3E92B
:100A1D0013F9E813F8DFF7EA28FAEB39FB8A408B74
:100A2D004150067BFF8B408B41C3EB94025002D2A9
:100A3D00673069047F0341617892E6FFC3E537941F
:100A4D008240110FC3E53794A040010FC3EF940608
:100A5D0040027F057E06E541C4540FF9E541C454BB
:100A6D00F0F8E540C4540F28F8C3E89EFAE9940065
:100A7D00FB4009C3EA9402EB940050047A02E4FBB4
:100A8D0041DBAA40AB41EBC4FEEAC4540F4EFCC39C
:100A9D00EA9CFAEB9400FBC3E813C313F8EA28FAB7
:100AAD00EB3400FB8A408B41C3EB94024002C267DA
:100ABD007806EBC4FE7B00EAC4540F4EFAC3EA98E5
:100ACD00FA4005C3940250027A027892E6FF306034
:100ADD000241DB855256855357D26043E680C3E40D
:100AED009AF8E49BF93067026175E8FAE9FBD3E9FE
:100AFD0013FDE813FC88528953C3EF94036038EF5C
:100B0D0020E00DE82CF8E93DF9ECFAEDFB020B3095
:100B1D00E828F8E939F9C3E82402F8E93400F97A4C
:100B2D00FE7BFFC3EF9403400E8A548B55884E898C
:100B3D004F8C508D5161A9885489558A4E8B4F8C9D
:100B4D00508D51306920C3E53394034019E542A21D
:100B5D00E713F8E555F4240138400B20E7087554E8
:100B6D00FFF42401F55561A9E8FAD3E813FC885286
:100B7D00C3EF94036020EF20E007E82CF8ECFA6156
:100B8D0095E8282402F87AFEC3EF940340088A54AE
:100B9D00884E8C5061A988548A4E8C50E56BC333B6
:100BAD005002646BF56B30600261B3753402D26034
:100BBD0043E680E52D54066026A840A941C3E913FC
:100BCD00F9E813F8C2AF53E67F759100C3E498F5C9
:100BDD0094E499F595759104D26043E680D2AF22E5
:100BED00D265754400752000306B03752040020CF2
:100BFD000CD265754400752040306B03752000D212
:100C0D00AF7801206722E52D54066002C265C3E569
:100C1D0041940540137802940540087803940540EB
:100C2D00027806306902780A206019E544601530B3
:100C3D00690AC3E53394034003D53406D2AFD26CB1
:100C4D0081DE71BBD2AF0000C2AF206726E541C384
:100C5D00FB940F40027B0FEB240530730123306AA8
:0F0C6D0002742820620123F93069027982E58B35
:100C7C00C39940B50544E59BF45440B5200281C8A6
:100C8C0030690A08C3E8940A4001088135206502DE
:100C9C00810CC26553E67F75910030671075940026
:100CAC007595FE759104D26043E680810CAE40AF21
:100CBC0041C3E49EF594E49FF59581AFC3E533946D
:100CCC00025002810C306502810CD80281DC813526
:100CDC00C26C53E67F75910085549485559575913A
:100CEC0004854E56854F57D26043E680D2AFE52D32
:100CFC0054066008206A020533020D18306C0D2072
:100D0C006B0A206507158115810215832278003046
:100D1C0064053065027801E53775F007A4F9E5F054
:100D2C0028F5F0E9A2F013A2F113A2F213F537C3E0
:100D3C0094785003753778C3E53795384008D266F8
:100D4C00C283C294C295306002A15285505685511F
:100D5C0057D26043E68022207D11C2AF754302C298
:100D6C0082D280D2AF759F43020F32C2AF7543025D
:100D7C00C282D297D2AF759F43020F32307243209A
:100D8C007D20C2AF75430390014A757E04C295C2A3
:100D9C0097306204D294A1A6D282D2AF759F53022F
:100DAC000F32C2AF75430390014A757E04C283C2F1
:100DBC0080306204D294A1C6D282D2AF759F330226
:100DCC000F32207D17C2AF754303900125C29530B9
:100DDC006202D294D2AF759F53020F32C2AF7543E9
:100DEC0003900125C283306202D294D2AF759F3337
:100DFC00020F32207D11C2AF754304C280D297D24C
:100E0C00AF759F33020F32C2AF754304C297D280C5
:100E1C00D2AF759F53020F32307243207D20C2AF88
:100E2C00754305900139757E01C294C2823062040B
:100E3C00D283C142D280D2AF759F43020F32C2AF70
:100E4C0075430590015B757E80C294C2823062044A
:100E5C00D295C162D297D2AF759F43020F32207DDB
:100E6C0017C2AF75430590011BC294306202D28346
:100E7C00D2AF759F43020F32C2AF75430590012F5D
:100E8C00C2943062EBD295D2AF759F43020F3220E1
:100E9C007D11C2AF754306C297D282D2AF759F53F4
:100EAC00020F32C2AF754306C280D282D2AF759F99
:100EBC0033020F32307242207D20C2AF7543019055
:100ECC00015B757E80C283C280306204D295C1DE24
:100EDC00D297D2AF759F33020F32C2AF75430190D8
:100EEC000139757E01C295C297306204D283C1FE6E
:100EFC00D280D2AF759F53E132207D16C2AF7543BD
:100F0C000190012FC283306202D295D2AF759F330C
:100F1C00E132C2AF75430190011BC295306202D21F
:100F2C0083D2AF759F53C26622900119757E00C2A1
:100F3C0083C294C295C280C282C297C26222788058
:100F4C0076090876090876040876FF087603087691
:100F5C00FF087609087603087601087601788C7606
:100F6C00010876FF0876FF0876FF0876FF0876FF03
:100F7C000876030876FF0876FF0876FF08762508C2
:100F8C0076D00876280876500876040876FF08761E
:100F9C000208760008767A0876FF08760108760152
:100FAC00087600087603227887E6FFC272BF030238
:100FBC00D2727888E6C394036008C27DE630E10201
:100FCC00D27DC27E7889E630E102D27EC3EF9402F4
:100FDC006008758E01D273020FEB758E00C27322FE
:100FEC007880E6149000809378A4F67881E61490CB
:100FFC0000809378A5F67886E61490008D9378A6F9
:10100C00F6789CE67538FF75390CB402067538A075
:10101C0075390AB4030675388275390578A3E61458
:10102C0090009A93F569120F3522227896E6FA7899
:10103C0097E6FB7888E6B40305C3EB940EFB307F90
:10104C00047A007BFFC3EB9AFCC3948250027C822F
:10105C007575000575EC8575F0A4C3E5F0947D40BD
:0F106C00F222D27F11371205B47A007B007C107C
:10107B001205AAE55F2AFA74003BFBDCF37C04C380
:10108B00EB13FBEA13FADCF7FEC27F113722E5EF15
:10109B0020E6037520000520903FFFE52014600635
:1010AB00901DFF1460009304600375EF1253D9BFBA
:1010BB007581C043FF801205A575EF0243B203E5AE
:1010CB00B3240420E70DF521E5E320E0068521B3E9
:1010DB0043E301120F357580F275A40D75F13F7561
:1010EB00D4DF75904F75A5B075F2F075D50075A668
:1010FB000175E241E4F8F6D8FD756B01120F4A1247
:10110B0015C578988676753001C2AF1205BE1205EB
:10111B00CE1205B41205D51205B41205DC1205B4B6
:10112B00C2AF78FA79FA308507D9FBD8F7021C00E1
:10113B00120FB3120FEC1136113778988676120F07
:10114B003575885075891275C82475910475D8400A
:10115B0075A82275B80275E690759B80759D007514
:10116B00D10E75BC5875BB0975BA1175E88012059F
:10117B00A5D2AF1208B353DACF207E0343DA203067
:10118B007E0343DA1043DA01C2D8C2711205BED214
:10119B00617B037A0CE55E70077A0CDB0302112B83
:1011AB001205B420700302112BC270E55FC39402C9
:1011BB0040E1E52F541F856160F561B560D5DAD547
:1011CB00C26153DACF207E0343DA20307E0343DA49
:1011DB0010C2D8C27178A2E67008D274E52F54E021
:1011EB00F52FC2757529001205B9307409C3E529AD
:1011FB00940A4002D2751205AA7802307402780064
:10120B00C3E55F9840F0C2AF1205CE1205CE1205B2
:10121B00CED2AF1205BE754D007888E6B4030261DD
:10122B00021205AA788CE6C394015003021302E55F
:10123B0030C394015003021302207435C3E55F944D
:10124B00FF5003021302C2AF1205E3D2AF1205B96E
:10125B00C3E55F940150EFC2AF1205CE1205AF127A
:10126B0005CED2AF1205B9C3E55F94FF40E9021773
:10127B006D7F02D27F11371205B9C2AFC27F113712
:10128B00AE5FC3E55F947FD2AF40761205A5C2AFC8
:10129B001205E3D2AFDFDC116EC3EE94057897F63F
:1012AB001205BE1216071216F07F0AD27F113712E3
:1012BB0005B9C2AFC27F1137AE5FC3E55F947FD272
:1012CB00AF50E61205A5C2AF1205CE1205AF12053F
:1012DB00CED2AFDFD6116EEE24057896F61205BE90
:1012EB0012160712171F1205B91137C3E55F94FFCA
:1012FB005002414402176DC3E55F954D4003855F76
:10130B004D1205B978017988E7B403027805C3E576
:10131B005F9840024124C2AF1205E31205E31205A8
:10132B00E3D2AF1205BE753000E4F531F53205316D
:10133B00E531F470390532789AE678191460127831
:10134B003214600D787D14600878FA1460037532DE
:10135B0000C3E53298401715327531B4789986760B
:10136B00C2AF1205E3D2AF789886761205B9120593
:10137B00AFE52A7005307402212B780120740278B6
:10138B0006C3E55F9840A77888E6C3940360031211
:10139B0005B9E52A700302112BC2AF120F35E4F524
:1013AB0022F523F524F525F526F56AD2AF7885E6E7
:1013BB00C333F568E4F545F546F547F548F549F5CA
:1013CB0073F52CF52DF53775730875BB101205A544
:1013DB001208B7E5E820ECFBA8BDA9BEE97001F83F
:1013EB0088741208BB75730875BB107887E6FE7698
:1013FB0002120FB37887EEF6C2AF7564FF12095372
:10140B00852264852265852266D2AF7522017524FB
:10141B000175250175260185636C756D017888E66C
:10142B00B40307C27D307602D27DD268D2697533A0
:10143B0000120E9B120EC012097312097A12097355
:10144B0012097A120973021461C2AF120FB3D2AF31
:10145B0075730075BB09120BFE1206AE120D191235
:0E146B000D6312097A120BED306D0312070AA1
:1014790020670312085630670312089D120D1912CE
:101489000D8812097A120BFE306D0312073F120DF7
:1014990019120DFF12097A120BED306D0312079D17
:1014A900120D19120E2412097A120BFE306D031255
:1014B90007FA120D19120E9B12097A1208B7120BAC
:1014C900ED120D19120EC01208BB12097A306935D6
:1014D900206B3285676485676585636C756D0179F5
:1014E900187A0CC3E53399400FC269D26A8A3585E7
:1014F900676485676602150EC3E55F9401400302C0
:10150900146102158B306A1B206B18E535147004C1
:10151900C26A8154F535C3E55F9401400302146141
:1015290002158B753600C3E56278FA985054307409
:1015390004E52A604D7888E6B40317207D052076F6
:1015490007A15B307602A15B206B07D26B856764CC
:1015590081A078F0306B058567647820C3E54198F0
:1015690050028161306B1BC26BC27D307602D27D25
:10157900D26A75351285676481610536E55F600257
:10158900A18E753600C2AF120F357887E6FE760256
:10159900120FB37887EEF6E4F522F523F524F52545
:1015A900F526F568C268D2AF1205A5120F35307459
:1015B90009C3E53694054002212B6134901A0D7850
:1015C90020121649E520B4550CA3121649E520B49A
:1015D900AA030215E7120F4A121607021606901AF5
:1015E9000378807B0A121649A308DBF9901A0F7851
:1015F9008C7B18121649A308DBF9901A2722C2AF6F
:10160900121688121662901A00740E12164EA374DE
:101619000412164EA3741412164E901A0378807B86
:101629000A12164DA308DBF9901A0F788C7B181251
:10163900164DA308DBF912169B121679901A272268
:10164900E493F622E6438F01538FFD75EF0275B7D8
:10165900A575B7F1F0538FFE22438F02438F0175B1
:10166900EF0275B7A575B7F1901A0DF0538FFC22EB
:10167900901A0D7455D14E901A0E74AAD14E227A31
:101689003079D07820901A40D149E520F709A3DABA
:10169900F7227A3079D0901A40E7D14E09A3DAF9C6
:1016A90022AB77A878BB01027980BB02027981BBA2
:1016B90003027982BB04027984BB05027986BB06E1
:1016C900027992BB07027987BB080279A3BB090299
:1016D900799CBB0A027988BB0B027989E8F7227CDD
:1016E900051205BEDCFB22C2AF1205CE1205D512CA
:1016F90005DC1205E31205AF1205CE1205D5120558
:10170900DC1205E31205AF1205CE1205D51205DC70
:101719001205E3D2AF22C2AF1205E31205DC1205AE
:10172900D51205CE1205AF1205E31205DC1205D557
:101739001205CE1205AF1205E31205DC1205D5120A
:1017490005CED2AF22AE77AF78C2AF1205CE120561
:10175900CE1205CE1205AFDEF21205E31205AFDF98
:10176900F8D2AF22D1F0D1E8D1E8757701757801C7
:10177900757900F14E7C05AD5F1205BEC3ED955F2D
:1017890070F5C3E55F9401400AC3E55F94FF4032F9
:101799000217A9D1AAD107D1F0C2AF75EF12D1E8CA
:1017A900DCD50579C3E5799403500280C6D1E805F3
:1017B90078E5771490009F93F808C3E5789850026C
:1017C90080AED1E8D1E80577C3E577940C50028063
:0D17D9009C120F4AD107C2AF75EF12D1E884
:0319FD000210993C
:101A00000E0414090904FF03FF0903010155AA018B
:101A1000FFFFFFFFFF03FFFFFF25D0285004FF0259
:081A2000007AFF01010003FF41
:101A400023416C69676E424C333558232020202097
:101A500023424C48454C4923463333302320202031
:101A60002020202020202020202020202020202076
:101C0000C2AFC2D353D9BF7581C043B20343FF8073
:101C1000752438752503B1C975EF0275E24043F1AB
:101C20002053A4DF75D400D2857DFA780379E67C51
:101C300010752200752300901DD67B0675249875BB
:101C400025013085028142208508D8FBD9F9DCF7CF
:101C500081B4308508D8FBD9F9DCF781B4B189E4C7
:101C600093A3C39A6004DDC381B4DBDBB17B600264
:101C7000812B7B08E493FAA3B15CDBF87A30B15C8A
:101C8000752200752300B17BEAFCEBFDC3ED94FEE9
:101C9000400EB17B8A278B28ED30E0048A828B834B
:101CA000B17B7AC270D8C3ED94FE601350CEBD00F4
:101CB00025EC60097520007521FF0200008100A855
:101CC00027A9280809D804D90281D3B17FEA89AAB3
:101CD000F281C50D81A0C3ED94035049EDA2E092BD
:101CE000007AC5C3E5829400E583941C50902000DF
:101CF00010438F02438F0175B7A575B7F1F030001F
:101D00001FA827A9280809438F01538FFDD804D99C
:101D100002A12089AAE275B7A575B7F1F0A3A10DBC
:101D2000538FFC817C7AC1BD030CE493A3FAB140CC
:101D3000DCF8B138817C817EAA22AB23B15CEBFA5E
:101D4000EA6222752608C3E52313F523E52213F57D
:101D50002250066323A0632201D526EAB1C9B1C986
:101D600075260AEAF4200102D285300102C285B14B
:101D7000C9C3134002C201D526EB22B17FEAFB2082
:101D80008502A17F308502A184752608AE24AF2587
:101D9000C3EF13FFEE13FEB1CDB1C9C3EA13308513
:101DA000024480FA30E703632201C3E52313F523DD
:101DB000E52213F52250066323A0632201D526D91C
:101DC000E52265236523F52222AE24AF250E0FDE22
:101DD000FEDFFCD20122424C48656C693437316326
:041DE000F3300601D5
:00000001FF
